:10000000BFC1D8C1D7C1D6C1D5C1D4C1D3C1D2C156
:10001000D1C1D0C1CFC1CEC1CDC1CCC192C3CAC1A3
:10002000C9C1C8C1C7C1C6C1C5C1C4C1C3C1C2C19C
:10003000C1C1C0C1BFC131E1FBCF867C000080C01F
:100040000993DFFFFFFEA8760BE03A0001FE0000F7
:100050000380DFFFC7FF7C0000058FEF9FFFCF9677
:1000600060107C0000FE1060303CC00E8FFFFFFF70
:10007000E87203C07001FEBC020FC0F801F07DC839
:10008000A3FC0F339234FF0F7FFF69AA9040E00179
:100090000DE50031FD037FE111EFFFFF81DC21C0A1
:1000A00006FE03F0FB8312301039E3C3BFB8F3D070
:1000B0000661C3FCE4FC7FF9C01CC0C03E007C4C60
:1000C00098FE07C13DF07F8FDDCCC19838E11C7CE4
:1000D000C85F07F1C6003C07EC1E73F02BFFF5B5B7
:1000E0006AAAA222491249249492525252952A0095
:1000F00000000002AB56B5B5B5B6D6AD5AB56AD557
:100100006AB55AAD55AAB555AAAB55556AAAAAAA59
:10011000B555555554AAAAAAAA955552AAA5552A25
:100120009552A552A54A952A54A94A952A54A954EC
:10013000AA552A9554AAAA00000000000000AAAA05
:10014000B5556AAAD556AAD556AAD55AAB556AADA1
:1001500055AAB556AAD55AAB555AAAD556AAAD55E1
:1001600056AAAAD555556AAAAAAAAAAB5555555555
:100170002AAAAAAAAAAA5555552AAAA955552AAA09
:100180009540000306090C101316191C1F22252880
:100190002B2E313336393C3F414447494C4E515365
:1001A00055585A5C5E60626466686A6B6D6F707108
:1001B0007374757678797A7A7B7C7D7D7E7E7E7F9E
:1001C0007F7F7F7F7F7F7E7E7E7D7D7C7B7A7A795D
:1001D000787675747371706F6D6B6A68666462604F
:1001E0005E5C5A585553514E4C494744413F3C3947
:1001F0003633312E2B2825221F1C191613100C09FB
:10020000060300FDFAF7F4F0EDEAE7E4E1DEDBD8FF
:10021000D5D2CFCDCAC7C4C1BFBCB9B7B4B2AFADD8
:10022000ABA8A6A4A2A09E9C9A9896959391908F15
:100230008D8C8B8A8887868685848383828282815F
:100240008181818181818282828383848586868780
:10025000888A8B8C8D8F9091939596989A9C9EA06E
:10026000A2A4A6A8ABADAFB2B4B7B9BCBFC1C4C756
:10027000CACDCFD2D5D8DBDEE1E4E7EAEDF0F4F782
:10028000FAFD200022002400260028002B002D006B
:1002900030003300360039003C0040004400480084
:1002A0004C00510055005B00600066006C0072005D
:1002B00079008000880090009800A100AB00B50094
:1002C000C000CB00D700E400F20000010F011F01C5
:1002D0003001430156016A0180019601AF01C80156
:1002E000E30100021E023F0261028502AB02D4025A
:1002F000FF022D035D039003C70300043D047D044A
:10030000C2040A055705A805FE055906BA062107C5
:100310008D0700087A08FB088309140AAE0A500BFF
:10032000FD0BB30C740D410E1A0F0010F410F611F2
:10033000071329145C15A116F9176619E91A821C0E
:10034000341E0020E721EB230E265128B72A412D29
:10035000F22FCC32D1350439683C0040CE43D64729
:100360001C4CA3506E55825AE45F9865A26B0972CB
:10037000D17800809C87AD8F389845A1DCAA05B55F
:1003800011241FBECFE5D4E0DEBFCDBF11E0A0E059
:10039000B1E0E4ECF4E102C005900D92A43AB1079B
:1003A000D9F711E0A4EAB1E001C01D92A93BB10761
:1003B000E1F793C125CE682F80E02091A001309114
:1003C000A1012115310531F4C901613021F581E028
:1003D00090E0089561506F3FE9F02091A4014091B1
:1003E000A2015091A301322F3078220F41F4FA017B
:1003F0004F5F5F4F2491322F3078220F2160880F9A
:1004000031118160615078F75093A3014093A201AC
:100410002093A40199270895CF93DF9320E06150A2
:100420006F3F19F19927EC01CB55DE4FDC01A80F86
:10043000B91FA355BE4F8881982F9078880F888365
:10044000882371F48D919C911197FC0101968D93F5
:100450009C9311978491982F9078880F816088835E
:10046000220F91112160615030F7822F9927DF917F
:10047000CF910895CF92DF92EF92FF920F931F9347
:10048000CF93DF938091A901882309F0BBC08091AD
:10049000B801882309F03CC025EAC22E21E0D22E03
:1004A000C0E0D1E003E09DEAE92E91E0F92E81E081
:1004B00082DF882319F087E07EDF8A8F81E07BDF8F
:1004C000882321F085E077DF80518B8F8A8DE82F9C
:1004D000FF27EE0FFF1FEE5AF74F85919491F7011A
:1004E000819391937F01F60111926F010150A096C3
:1004F00007FFDDCF8091A0019091A101009729F025
:1005000001979093A1018093A00180E28093B801AC
:100510008091B80181508093B80100E0C0E0D1E043
:100520008FE0F82E61E0802F77DF882319F067E0F5
:10053000802F72DF182F61E0802F6EDF882319F083
:1005400068E0802F69DF482F112311F08B8D180F81
:10055000988D998F8F89888F8E898F8B1E8B112311
:1005600029F48E858823D9F0192FF82E1123B9F09C
:100570001C8F188A198A19821A821A861B86FF0C08
:10058000FF0CFF0CFF0CFC868B81E82FFF27EE0F82
:10059000FF1FE058FE4F808191818C8B9D8B842FB3
:1005A00082958F70942F9F70FE01E80FF11D90834C
:1005B000863021F49295907F9E831CC08A3019F476
:1005C0001C8A1D8A17C08B3011F41D8E13C08C300D
:1005D00021F49295907F9C870DC08D3059F4417025
:1005E00091FF03C066E370E002C06CED70E086EA44
:1005F00090E099D00F5FA096043008F491CF86E088
:100600008093A9018091A90181508093A901A0E064
:10061000B1E003E0FD018485C82FDD278181608979
:100620007189680F711D8281681B7109608B718BE4
:100630008285E82FFF27EE0FFF1FE058FE4F8081D5
:100640009181C81BD90BD7FF02C0C0E0D0E0FD01EB
:10065000C487848DE82FFF27EE0FFF1FEE57FD4F55
:1006600045915491FD0113851123A9F0858DE82F43
:10067000FF27EE57FE4F8491282F332727FD309513
:1006800088E090E0811B910902C0359527958A95F5
:10069000E2F7420F531F460F571FFD01428B538B4A
:1006A000C68F858D9581890F858F8489958900975F
:1006B00039F00197848B958B892B11F48481828783
:1006C0000150909607FFA6CFDF91CF911F910F9118
:1006D000FF90EF90DF90CF900895CFE5D4E0DEBF9C
:1006E000CDBF31E0832E992480E88BB98FEF8AB992
:1006F0008FE097E290938900809388009092800029
:100700008AE08093810084EB87BD82E080936E0055
:1007100084BD85BC84B885B87894B19BFECF82E057
:1007200086BBA8DEFACF1092AB01A12C6093B60174
:100730007093B70160E16093AA014EBB8093AB0157
:1007400008950F920FB60F921F921F932F937F93CE
:100750008F939F93EF93FF931091B5011BB9109165
:10076000AA01AA0C89F48091AB018150B8F0809362
:10077000AB01E091B601F091B701A590E093B6010D
:10078000F093B7010894AA1C20F4139515FD1FE1FE
:1007900003C0115008F411271093AA011051F09BC7
:1007A000110F20911201220E20911301321E732D80
:1007B00077FD709576957695705120911E017203A4
:1007C000110D20913201420E20913301521E2091D1
:1007D000260178E0521608F4719520913E017203CB
:1007E000110D20915201620E20915301721E209131
:1007F000460178E0721608F4719520915E0172034B
:10080000110D21E0880C991C97FC822696FC82260B
:1008100080917C0186958695869525E0281B782D0C
:100820007F7375FD706C72030594702D20917E01AD
:100830007203110D10581093B501FF91EF919F9124
:100840008F917F912F911F911F900F900FBE0F904E
:100850001895BA0AC20AE00AFF0A200B400B580B8F
:10086000660B7D0B8B0B9D0BB10BCF0BED0B090CAE
:10087000200C2B0C450C660C870CA30CBF0CDD0C5C
:10088000FA0C100D2F0D4E0D6C0D880DA90DC40D19
:10089000E20D020E190E2D0E4D0E610E790E950E03
:1008A000B30ECE0EF20E100F2A0F4D0F710F990FCF
:1008B000C30FE90F001022103D1055106B1081106E
:1008C0009710AD10C310D910EF10051116112C118F
:1008D000421158116E118411A311BE11D411DE11F1
:1008E000F6110212171222123412491262127712F2
:1008F0008912A012B512C612DB12E712FE120E13F5
:10090000351354137C138B13AA13D513FC131B1428
:1009100033145214701486149C14AE140090F0001A
:10092000000002301228D0492381208F01020914CF
:100930001024906093C21012885160954302590EA2
:10094000097440261120994502691609D618DE4817
:10095000311ACAA18E0320136C9048338062814EF5
:1009600033614A9CC32592D74823141252A451AA3A
:100970004C092472884DA3D46AB4820541252A45C6
:1009800004A1C09241A0049A101288559A992A860F
:100990005A29D2C8759A992E885A2A130895AA9D61
:1009A000328A5B09A45ADD529D61A01BE906653AB3
:1009B000CB20AC05802E01484D9584878B0AB4EE80
:1009C0000C0DC48310538C7019003246D0CA14E346
:1009D000340A719B02730C964AAD208C50494E919B
:1009E00046A9302491CA21368F51AAD20815049401
:1009F000E9141287024906801268415C9442ACD423
:100A0000C95432D14E9643ACD4C97442D1509844A3
:100A1000AD54E99452D87022D6EA967B4170AC1A54
:100A20002655A5FA4B9C2B0D34D74AF2DD45C29CC6
:100A3000CB557A1BE4AF94C5F00BF6D98622E1586A
:100A400031CCAB4BF217380D32574DB30CA5C2B4B5
:100A500066995617E32EF0AE3BCB5E375218462808
:100A600024A748A354981248E512A5368F51AA121C
:100A700008150494E91412870A94920D0024D08278
:100A8000AD288559A992A865A2A12C8759A992E8F9
:100A900085A36D30895AA9D328A5B2A59FE71B85E8
:100AA0005A91CA21C55EDA630895AE1589E45301EF
:100AB0005A9F613055CE461B656200000000000061
:100AC0000000BFB42BAD9B465FAF576BD3817E1B3D
:100AD0003702E00D9805B0B838176702FCE06000F7
:100AE0001B306A3017EBD5F9C0C0097B81881C85A3
:100AF000931C380630C438184702FCE05D9C00C0E7
:100B0000B417E2F4E0621B34BDC4C43877A6CF0149
:100B100088C6188308E06486CCC218C70324E000A6
:100B2000CB198338E0639C0BF180308E05D84B1ACB
:100B30008BBE409635177C412C6A2EF84258D40063
:100B4000B8B401682E03905D8720BB0E41741C82EF
:100B5000E03905B06CCB1380B18A967101B3000007
:100B60001A2000000000B8B401682E03905D8720B1
:100B7000BB0E41741C82EC3905E86CCBB0BD8A8594
:100B8000F86CC0000000001A201A40BF1801C430E1
:100B900003885F8BD0E2344DA000000000BD17E158
:100BA000C02FC3885D8710B68A1701B301A2000069
:100BB00000BD01802FCE45E9C4BB38174702E0E0F5
:100BC0005BAE16EB85BAE16EB85B8694B80E20BFBB
:100BD000B42BAD9B465FAF576BD3817E1B3702E0D2
:100BE0000D9805D8BA3816C702CCE05A0000B3B445
:100BF0001681C02D8E05C00690BDB2176702E0E0D9
:100C00005F8BD34976702E0DA0000690BF17A70208
:100C1000ECE05C1B41A4B60D21706D068402EC0073
:100C2000B8034200DA0000000000009402454027AB
:100C30008D2D01A59B0E012800280E04D9C0A314F8
:100C400042813C9B009903494A69264D2518A534E9
:100C500093269294D24C81A4A5349406928C529AF5
:100C60004993493669009003492E70270E04F09C81
:100C70003492069250E04901A4993493C692804F71
:100C80001A4A23494A6900971467028CD24B9A4A40
:100C9000114669278E04B81A4971320692680D24EC
:100CA000D81A4090013870240E04D89C3493C69210
:100CB00080E04F1C0920349280692580D24B009738
:100CC00003493C7029C0528684A3349446926CD266
:100CD0005109B3494E6866CD2559A1AE009C120654
:100CE0009240D2481A49C12069240D2481A49E1241
:100CF00041A42503484B0690920097014670278E29
:100D00000538A51467025CD24D809D013E02880023
:100D10009914A1A1280D2529A4A0349362704F0134
:100D2000A4AA3494A692A8529A49E349326900973A
:100D3000349460278D24D9A4971326926CD24E0642
:100D400088AC3495E692B0550A83494E6900A514E3
:100D50000264E051A914A2804C9C0A03814E2884AD
:100D6000D9C0A23814E2884D9C09F3809402454012
:100D7000278D2D01A59B0E0128026C519C0AC38171
:100D8000542C55EAE5529D448F024536264D2CD908
:100D9000A58F0E012C6926CD24E1A4993493669287
:100DA0005C4C9A4963492E6900AC1702D8D2599A13
:100DB0004B115E2A8538A014A28C5109E1366926B0
:100DC0004D24B9A49F34956029C511A49F1406929F
:100DD00088D25001A4AC1542B0D2539A4A33494E3E
:100DE0006900AD14A270D2529A4AD1582B4578B1FD
:100DF0003495669294D2539A4A33494A69288D258C
:100E000019A4C7983C0D1863B1988C63818E1C8718
:100E100002FC034400000621A101C02D166B15A1A0
:100E2000C0B80E41761C81C000162000000C0E6375
:100E300048181C86902F4E0601C0C2DA348185CC3A
:100E400069030B90D20611C0BF3818C700C4DA344A
:100E50008189CC69031390D2062711A400000000F9
:100E60000000B61701C02ECE05E868800161780049
:100E7000BB3817E7030368D20099E814A51A945207
:100E800089914BD129452F409914A29452A9533DE1
:100E90002294528A5099E814A51A9452899E914A34
:100EA0002954AA5E9132297A0528A5E8132297A031
:100EB000528A5099E814A51A9452899E914A29455C
:100EC0002899E814A29452899E914A29452899E8C4
:100ED00014A51A9452899E914A29452F4E9533D2D2
:100EE000297A052F40A5E914AA552F48A5E814BD75
:100EF0002A5099E814A51A9452899E914A29452F9F
:100F00004499E814A29452A9533D229452F48A5071
:100F100099E814A51A945289914BD029452F4099EC
:100F200014A2945289914A26452899E814A51A9743
:100F3000A05289914BD12954AA5E994A297A052F4A
:100F400042954BD226452F48A5E894BD1099E91447
:100F5000A51A97A052F4099E914A297A052F409923
:100F6000E914A297A052F4099E914BD0297A052F3B
:100F70004099E914BD051A97A14AA5E8133D2297A7
:100F8000A052F40A5E8133D229452F40A5E8133DD3
:100F90002297A052F41D0A5E9899E914BD051A978C
:100FA000A14AA5E9133D0297A052F48A5E8133D08D
:100FB000297A452F40A5E83A133D2297A052F49D87
:100FC0000A5E8099E814BD251A97A052F4099E91F3
:100FD0004A297A452F4099E914A297A481D2F4C9ED
:100FE0009E814BD2297A052F409914A51A945289D3
:100FF000914A2945289914A2945289914A26452854
:1010000099E93A74BD051A97A252F449914A2954B4
:10101000AA5E852F4267A452F40A5E82874BD000F5
:10102000000099E814A51A9452899E814A294528FE
:1010300099E814A29452899E814A264528C499BCF5
:10104000B762D05D8C41762D05D8C617A2D85E8CCC
:10105000617A2D85E8C717E2EC5F8C717E2EC5F8AA
:10106000C617E2DC5F8C616E2E85F8C417A2D05ED5
:101070008C417A2D05E8C617A2D85E8C617A2D8541
:10108000E8C717E2D85F8C717E2D85F8C71802E09B
:10109000600C71802E0600C61802E0600C61802E84
:1010A0000600C617E2DC5F8C617E2DC5F8C41762AE
:1010B000D05D8C41762D05D8C41762D05D8C417609
:1010C0002D05D8C617E2DC5F8C617E2DC5F8C617EA
:1010D000E2DC5F8C617E2DC5F8C717E2E05F8C9182
:1010E0007E2E05F8CB17E2E05F8C917E2EC5C0CB3B
:1010F00018C3105F8CB18C3105F8CB18C3105F8C0E
:10110000B18C3105F8CB18C30C5F8BA16E2CC57068
:10111000A70348000000C41742C45D0C21742C458D
:10112000D0C21742C45D0C01742C45D0C016C2BC9D
:101130005B0BF16C2BC5B0BF16C2BC5B0BD16C2B2B
:10114000C5B0BD16E2B85B8BB16E2B85B8BB16621D
:10115000B8598BF1662AC598C617E2DC5F8C617EB0
:101160002DC5F8C717E2E05F8C717E2E05F8C9180F
:1011700002E4600C91802E4600C717E2DC5F8C61B0
:101180007E2DC5F8BD017E300E4611C4C03817E76C
:1011900002F4E05DAE976BA5DAE976BA5DAE8DA19B
:1011A000701C40B80034989A6C4D3621C0C40E00B3
:1011B000170696E0E05C1C0B8368D282CE00588054
:1011C000015DC4D0B6A0348183144530B6800600DA
:1011D0000BF036A00006840001A400000000BF8AC6
:1011E000A2B800001A42FC600C2DA017BA2001A37F
:1011F0002F6308C5FED00006840001A40000BF01D3
:101200007A00BB00DA0D217E001A42EB680005B0BF
:101210000B18AA2B67B400780006840000000000B9
:101220001A20588000C4D08034818C1B40031CD20B
:1012300006481B40000000000B3B416A2DCE05C153
:10124000C0BA38176702F4E000BFE6348E017FC8E9
:10125000702FF903805FF21C0BFE63680E00000024
:1012600000006D00C7E70D218DCD1A431003440621
:101270001006900BD0D280584000C4D08034818CAE
:101280001B40031CD205F81B40900E01201C02409D
:10129000380480700900E01201C024038048070070
:1012A000B8B400DA00D100017002E805D8694BB883
:1012B000AA2B7BB4000000BB01740002E0368D2530
:1012C000D4100BB34400BD36817601A402EC0005B6
:1012D000D001A11A4BA8AA2B77B4000001A20000EC
:1012E00000B8017602FC00BE8AA2B7E2F40342060F
:1012F0001001B40C000D1817F1545703680000BF1B
:10130000003423497A0002FC002445B01B20CBB0F6
:10131000A9189C43245C720CCD262F131388658D6D
:101320000E2193A4D7E462710C6171C431C62710F9
:10133000C417FC849099E814A51A9452899E914A86
:101340002954AA5E9132297A0528A5E8132297A08C
:10135000528A5286CBB0A9189C43245C720CCD26CD
:101360002F131388658D0E2193A4D7E462710C614D
:1013700071C431C62710C43C17FC8490C417E2E046
:101380005F8C41703100000000000099E814A51A3C
:101390009452899E914A29452F4499E814A2945267
:1013A000A9533D229452F48A528699E914BD051A34
:1013B00097A14AA5E9133D0297A052F48A5E8133B2
:1013C000D0297A452F40A5E83A133D2297A052F440
:1013D0009D0A5E828699E814BD251A97A052F409E9
:1013E0009E914A297A452F4099E914A297A481D267
:1013F000F4C99E814BD2297A052F414399E914A55E
:101400001A954AA5E9132297A0528A5E8933D029FA
:10141000452F44A5132294528A52869914A51A94F2
:101420005289914A2945289914A2945289914A26B1
:1014300045294399E914A51A954AA5E9132297A0CD
:10144000528A5E8933D0294528A5133D0294528AD9
:101450005286A5140264E051A914A2804C9C0A0390
:10146000814E2884D9C0963811E2584D9C08F380EB
:10147000C91802E0638C0170318600B81683005AE7
:101480000C01762E05D8C417E2F45C0C417E2F4582
:10149000C0C417E2F05C0C417E2F05C0B801883053
:1014A0008600BF17A2EC5D00BB017A02E800A01421
:1014B000E702A8E0560690000943812870250E0433
:0414C000A1C00000C7
:1014C4000000000000080000000000000000000010
:1014D4000000000000000000000000000000000008
:1014E40000000000000807000000000000000000E9
:1014F40000000000000000000000000000000000E8
:1015040000000003090803000000000000000000C0
:1015140000000000000000000000000000000000C7
:1015240000000001060000000000000000000000B0
:1015340000000000000000000000000000000000A7
:1015440000000100030007000F001F003F007F00A0
:10155400FF00FF01FF03FF07FF0FFF1FFF3FFFFF18
:0415640070001C09EE
:00000001FF
